:100000007E29AA01AC01AB000130A8002C082A020D
:10001000031D0C282B082902043003180130031992
:1000200002302805031D01307A298030A100FE30FE
:100030000921013009217530AA0030302129A101A0
:10004000A117B200FE30092132080929A601AD002E
:10005000AE01A01126080319A0150530A500273010
:10006000AC0010303F200330AC00E8303F20AC0142
:1000700064303F20AC010A303F202D084628AB00F9
:100080002E08AA002D08A90035212908A900A503DA
:100090000319A01126080319502825020318572810
:1000A0002908031DA011A0195728303E092908006E
:1000B000B000861106118316861106110F308605D1
:1000C00083123008A01882283E30AA0080302121F7
:1000D0003330AF0096201330AA00883021219620BB
:1000E000643020219620643020212230AF009620F9
:1000F000283081200C30812006308120A014300867
:1001000082282014AF00201C90280611033C031CF9
:10011000952895200730AA00D0302121031408002B
:100120002014FE3C0319A3280615201C2010861558
:100130000F3086052F08F03986048611AF0E20187F
:1001400096283230202130087A292016201E2012CD
:10015000A01AAE28A016E7200318D5280830AC0056
:10016000FB20AB0DAC0BB028201EE02005210121A7
:10017000201AD520DA202B0803107A292016201EF9
:100180002012201BC828FE39A800201703107A2946
:10019000A01BD028AF00A017E7200318D5282F08F0
:1001A000EE200318D528201E7A29E02005212013EF
:1001B000A013A01222088400270884178004E628D0
:1001C0002208840027098005841780050800DA20AA
:1001D0000521E02001212808A01A0138AB000830D1
:1001E000AC00AB0D0318DA20031CE020052101212F
:1001F000AC0BF128DA20052122088400270800052D
:10020000FF3E230884002409E328230884002408EF
:10021000DD28A11B5828080083178001840AFF3EAF
:10022000031D0D297A29AC01AB00FF30AB07031C7D
:10023000AC07031C7A290330AA00DF3021211529DD
:10024000AA01E83EA900AA09FC30031C2A29A90733
:1002500003182729A9070000AA0F272929183029E0
:10026000A91C3429000034290800AE01AD0110306A
:10027000AF002A0DAD0DAE0D2B08AD022C08031CEE
:100280002C0FAE0203184B292B08AD072C080318BE
:100290002C0FAE070310A90DAA0DAF0B39292908A1
:1002A0007A29AB00AC00AA010830AF00A90DAA0D55
:1002B0002B082A02031C5F292B08AA020314AC0D89
:1002C000AF0B56292C087A291030B300AA01A901D6
:1002D000B00CAF0C031C72292B08A9072C080318BB
:1002E0002C0FAA07AA0CA90CAE0CAD0CB30B6829F5
:1002F0002D087A298313831203130800A001073005
:100300009F00FE308A01582040308A0158200E306C
:100310008A0158200A308A0158200E308A0158205C
:1003200000308A01582000308A01582000308A01AC
:10033000582000308A01582000308A01582020308F
:10034000840060308A010D21A030840050308A0181
:100350000D212030840050308A010C218A011520A3
:1003600064308A0113218030A1008A011F2053309C
:100370008A01582063308A01582068308A01582049
:1003800065308A0158206D308A01582061308A0119
:10039000582074308A01582068308A01582065300E
:1003A0008A0158208A0158206B308A0158202E304B
:1003B0008A0158206E308A01582065308A01582001
:1003C00074308A0158208030A100C0308A011F207B
:1003D0004C308A01582044308A01582052308A011A
:1003E00058202D308A01582073308A0158206330FC
:1003F0008A01582068308A01582061308A015820CB
:100400006B308A01582065308A0158206C308A018F
:1004100058206B308A0158206C308A0158206F3088
:100420008A0158206B308A0158200530AC00DC303E
:100430008A0114218A01152086108A11432BD001CC
:100440008A111F235108B7000130D0008A111F23E1
:100450005108B8000230D0008A111F235108B9009A
:100460001130D0008A111F235108BA000800370844
:10047000BB008A114D223C08B7003808BB008A1126
:100480004D223C08B800B91339133908BB008A1152
:100490004D223C08B900BA130800BC013C143B1EB5
:1004A0003C10BC14BB1EBC103C153B1F3C11BC15C2
:1004B000BB1FBC113C08AF00B0010A30AB00AC015F
:1004C0008A016421BC003B12BB123B13BB133C08E6
:1004D0003B07BC0008004008A9000A308A015121EE
:1004E000BD003D08AF00B0010A30AB00AC018A018D
:1004F0006421B4002E08B50034084002BE003D0E51
:10050000F039BD003D083E07BF0008008030A10063
:10051000CB308A011F2055308A01582075308A015E
:10052000582072308A0158208A11051AAC2A1730D7
:1005300041028A1103189D2AC10A8030A100C030EF
:100540008A011F200230A60041088A0127208A1153
:10055000051AAC2A8A01A72A8A118519C32AC1085B
:100560008A110319B42AC1038030A100C0308A0166
:100570001F200230A60041088A0127208A11851910
:10058000C32A8A01BE2A8A11851AD02A8A11851A9D
:10059000CB2A8A01C62AC8308A0113218A11D22A9D
:1005A0008A01942A8030A100CB308A011F204D306F
:1005B0008A01582069308A0158206E308A015820FB
:1005C0008A11051AF82A3C3042028A110318E92AD6
:1005D000C20A8030A100C3308A011F200230A60069
:1005E00042088A0127208A11051AF82A8A01F32A6B
:1005F0008A1185190F2BC2088A110319002BC20317
:100600008030A100C3308A011F200230A6004208BA
:100610008A0127208A1185190F2B8A010A2B8A113A
:10062000851A1C2B8A11851A172B8A01122BC830A8
:100630008A0113218A111E2B8A01E02A0800053045
:10064000A2000130A7000530A3000230A400D03082
:100650008A01C02050088A01C0208A01A520D1004B
:1006600008000530A2000130A7000530A3000230C9
:10067000A400D1308A01C02052088A01C02053084A
:100680008A01BE2008001430D0008A011F235108BF
:10069000C5001530D0008A011F235108C60016304E
:1006A000D0008A011F235108C7001730D0008A01EB
:1006B0001F235108C8001830D0008A011F23510899
:1006C000CA001930D0008A011F235108C900203008
:1006D000D0008A011F235108CB002130D0008A01AD
:1006E0001F235108CC002230D0008A011F2351085B
:1006F000CD002330D0008A011F235108CE002430C2
:10070000D0008A011F235108CF008A011F228A01CD
:1007100037228030A1008A011F200230A60039084C
:100720008A0127203A308A0158200230A600380872
:100730008A0127203A308A0158200230A600370863
:100740008A01272020308A0158208A0158208A01F6
:1007500058208A0158200230A6003A088A01272032
:1007600000308A01582043308A0158208A11541CD5
:10077000F32B8030A100C0308A011F204C308A0149
:10078000582061308A0158206D308A01582070301D
:100790008A0158203A308A01582020308A01582096
:1007A00061308A0158208A0158206E308A01582011
:1007B00020308A0158202D308A0158204D308A017E
:1007C000582065308A0158206E308A0158207530D3
:1007D0008A0158202D308A015820831686108312F2
:1007E00086148A112C2C8030A100C0308A011F2071
:1007F0004C308A01582061308A0158206D308A01BE
:10080000582070308A0158203A308A015820203010
:100810008A01582075308A01582069308A01582091
:1008200074308A01582020308A0158202D308A01E6
:1008300058204D308A01582065308A0158206E308A
:100840008A01582075308A0158202D308A0158209D
:100850008316861083128610013054180301B600E7
:100860003908A9000F308A010120B6058A11031941
:100870005F2C013045028A11031D4D2C0130851B70
:100880000301B6000130D4180301B6058A1103191B
:100890004B2C5414D4148A115F2C390846020319C6
:1008A0000130031D0301B600380847020319013067
:1008B000031D0301B6058A1103195F2C54148A1114
:1008C000541C742C3908480203190130031D03011C
:1008D000B60038084A0203190130031D0301B605AA
:1008E0008A110319742C54108A11851F782CD41086
:1008F000013054180301B600013049020130031DD4
:100900000030B6058A110319972C39084B020319D8
:100910000130031D0301B60038084C0203190130F1
:10092000031D0301B6058A110319972C5414030102
:1009300054180130B600013049020130031D003067
:10094000B6058A110319C12C01304F028A11031D0B
:10095000AF2C8A11851FAD2C54108A11C12C390877
:100960004D0203190130031D0301B60038084E0281
:1009700003190130031D0301B6058A110319C12CA7
:1009800054108A11851AC62C8A11CD2C0130AC0066
:100990002C308A0114218A01852B8A11851AD22CC8
:1009A0008A01CD2C8A01152032308A011321803032
:1009B000A1008A011F202A308A01582020308A0194
:1009C000582054308A01582069308A0158206A30F2
:1009D0008A01582064308A01582020308A0158202A
:1009E00069308A0158206E308A01582073308A019C
:1009F000582074308A01582065308A0158206C30A4
:100A00008A0158208A01582065308A0158206E30AA
:100A10008A0158208030A100C0308A011F20203078
:100A20008A0158208A0158204C308A0158206930A8
:100A30008A01582063308A01582068308A01582082
:100A400074308A0158208A01582069308A01582060
:100A50006A308A01582064308A01582020308A0187
:100A6000582069308A0158206E308A01582073302E
:100A70008A01582074308A015820C4018A118519CE
:100A8000482D8A118519462D8A01412D8A11612D23
:100A90008A11851A552D8A11851A502D8A014B2DE0
:100AA000C8308A0113218A11122F32308A01132192
:100AB000C40A440A8A11031D5F2D8A01432B8A014F
:100AC0003E2D8A01152032308A0113218030A10089
:100AD0008A011F2020308A0158208A015820543072
:100AE0008A01582069308A0158206A308A015820CA
:100AF00064308A01582020308A01582069308A01E8
:100B000058206E308A01582073308A015820743082
:100B10008A01582065308A0158206C308A0158209B
:100B20008A01582065308A0158206E308A01582089
:100B30008030A100C0308A011F202A308A0158204D
:100B400020308A0158204C308A01582069308A01AF
:100B5000582063308A01582068308A015820743048
:100B60008A0158208A01582069308A0158206A3049
:100B70008A01582064308A01582020308A01582088
:100B800069308A0158206E308A01582073308A01FA
:100B9000582074308A015820C4018A11051AD72DB3
:100BA0008A11051AD52D8A01D02D8A01D22C8A11DD
:100BB0008519E12D8A118519DF2D8A01DA2D8A1117
:100BC000FA2D8A11851AEE2D8A11851AE92D8A01CE
:100BD000E42DC8308A0113218A15A22832308A01F7
:100BE0001321C40A440A8A11031DF82D8A01432BDC
:100BF0008A01CD2D8A01152032308A0113218030DF
:100C0000A1008A011F202A308A01582020308A0141
:100C100058204C308A01582044308A0158205230E4
:100C20008A01582020308A01582061308A015820DA
:100C300066308A01582073308A01582074308A0146
:100C4000582065308A0158206C308A0158208A016A
:100C5000582065308A0158206E308A015820203093
:100C60008A0158208030A100C0308A011F20203026
:100C70008A0158208A01582045308A01582078304E
:100C80008A01582069308A01582074308A0158201E
:100C900020308A0158208A0158208A0158208A0170
:100CA00058208A0158208A0158208A0158208A0138
:100CB00058208A0158208A015820C4018A11051A37
:100CC000682E8A11051A662E8A01612E8A01612D0D
:100CD0008A118519722E8A118519702E8A016B2E40
:100CE0008A118B2E8A11851A7F2E8A11851A7A2EE7
:100CF0008A01752EC8308A0113218A15D82C32300A
:100D00008A011321C40A440A8A11031D892E8A010B
:100D1000432B8A015E2E8A01152032308A0113216D
:100D20008030A1008A011F2020308A0158208A01CA
:100D300058204C308A01582044308A0158205230C3
:100D40008A01582020308A01582061308A015820B9
:100D500066308A01582073308A01582074308A0125
:100D6000582065308A0158206C308A0158208A0149
:100D7000582065308A0158206E308A015820203072
:100D80008A0158208030A100C0308A011F202A30FB
:100D90008A01582020308A01582045308A01582085
:100DA00078308A01582069308A01582074308A01CD
:100DB000582020308A0158208A0158208A01582062
:100DC0008A0158208A0158208A0158208A01582017
:100DD0008A0158208A0158208A015820C4018A11AA
:100DE000051AF92E8A11051AF72E8A01F22E8A01A8
:100DF000FA2D8A11851A062F8A11851A012F8A0168
:100E0000FC2EC8308A0113218A01432B32308A011B
:100E10001321C40A440A8A11031D102F8A01432B8F
:100E20008A01EF2E8A0115208A011F228A013722AA
:100E30008030A100C0308A011F200230A60039088E
:100E40008A0127203A308A0158200230A60038084B
:100E50008A0127203A308A0158200230A60037083C
:100E60008A0127208030A1008A011F2054308A0186
:100E7000582069308A0158206A308A01582064302D
:100E80008A0158203A308A01582020308A0158209F
:100E90008A0158208A0158208A0158208A01582046
:100EA0008A0158208A01582055308A015820723012
:100EB0008A01582065308A0158206E308A015820F6
:100EC0008A11051A782F173039028A110318692FF1
:100ED000B90A8030A100C0308A011F200230A6006C
:100EE00039088A0127208A11051A782F8A01732F61
:100EF0008A1185198F2FB9088A110319802FB90318
:100F00008030A100C0308A011F200230A6003908BD
:100F10008A0127208A1185198F2F8A018A2F8A1129
:100F2000851A9C2F8A11851A972F8A01922FC83013
:100F30008A0113218A119E2F8A01602F8030A1001F
:100F40008A011F2054308A01582069308A015820B4
:100F50006A308A01582064308A0158203A308A0168
:100F6000582020308A0158208A0158208A015820B0
:100F70008A0158204D308A01582069308A01582052
:100F80006E308A01582075308A01582074308A01E9
:100F9000582065308A0158206E308A0158208A1105
:100FA000051AE72F3C3038028A110318D82FB80AE7
:100FB0008030A100C3308A011F200230A60038080B
:100FC0008A0127208A11051AE72F8A01E22F8A1148
:100FD0008519FE2FB8088A110319EF2FB803803046
:100FE000A100C3308A011F200230A60038088A0100
:100FF00027208A118519FE2F8A01F92F8A15851A53
:101000000B288A15851A06288A150128C8308A01F6
:1010100013218A150D288A01CF2F8030A1008A0163
:101020001F2054308A01582069308A0158206A30C4
:101030008A01582064308A0158203A308A015820A9
:1010400020308A0158208A0158208A0158205330C4
:101050008A01582065308A01582063308A0158205F
:101060006F308A0158206E308A01582064308A011E
:10107000582065308A0158206E308A0158208A1520
:10108000051A57283C3037028A1503184828B70A32
:101090008030A100C6308A011F200230A600370828
:1010A0008A0127208A15051A57288A1552288A1579
:1010B00085196E28B7088A1503195F28B703803091
:1010C000A100C6308A011F200230A60037088A011D
:1010D00027208A1585196E288A1569288A15851A88
:1010E0007B288A15851A76288A157128C8308A01C6
:1010F00013218A157D288A153F283708C0008A01E8
:101100006B223F08B700D2013708D3008A01312390
:101110003808C0008A016B223F08B8000130D200B5
:101120003808D3008A0131233908C0008A016B22B4
:101130003F08B9000230D2003908D3008A013123B8
:101140008A01432B8A0115208030A1008A011F20CB
:1011500020308A0158204C308A01582044308A01BE
:10116000582052308A01582020308A015820673098
:101170008A01582065308A01582062308A0158203F
:1011800072308A01582075308A01582069308A01EE
:1011900058206B308A01582065308A0158206E3003
:1011A0008A0158203F308A01582020308A01582077
:1011B0008030A100C0308A011F2020308A015820D1
:1011C0008A0158208A0158208A0158208A01582013
:1011D0008A0158204A308A01582061308A015820FB
:1011E00020308A0158208A0158208A0158208A011B
:1011F00058208A0158208A0158208A0158208A01E3
:1012000058200130C3008A15051A36298030A10004
:10121000C0308A011F2020308A0158208A015820BE
:101220008A0158208A0158208A0158208A015820B2
:101230004A308A01582061308A01582020308A01C2
:1012400058208A0158208A0158208A0158208A0192
:1012500058208A0158208A0158208A0158200130DC
:10126000C3008A15051A36298A1531298A15851968
:1012700068298030A100C0308A011F2020308A01F7
:1012800058208A0158208A0158208A0158208A0152
:1012900058208A0158204E308A01582065308A0132
:1012A00058208A01582020308A0158208A0158206D
:1012B0008A0158208A0158208A0158208A01582022
:1012C0008A015820C3018A15851968298A1563295E
:1012D0008A15851A75298A15851A70298A156B2928
:1012E000C8308A0113218A1577298A150329053008
:1012F000A2000130A7000530A3000230A400D130C5
:101300008A01C02014308A01C02043088A01BE200F
:10131000C3088A15031DF3298A0115208030A10016
:101320008A011F2041308A01582061308A015820EB
:101330006E308A01582073308A01582063308A0148
:10134000582068308A01582061308A0158206B305B
:101350008A01582065308A0158206C308A01582053
:1013600074308A01582069308A0158206A308A0115
:10137000582064308A01582031308A0158203A3090
:101380008A0158201530D0008A011F235108C1005E
:101390008030A100C0308A011F200230A600410821
:1013A0008A0127203A308A0158201630D0008A015D
:1013B0001F235108C2008030A100C3308A011F20C2
:1013C0000230A60042088A0127208A0186221530B1
:1013D000D2004108D3008A0131231630D2004208DE
:1013E000D3008A0131238A0115208030A1008A01AF
:1013F0001F2055308A01582069308A0158207430E6
:101400008A01582073308A01582063308A0158209D
:1014100068308A01582061308A0158206B308A0177
:10142000582065308A0158206C308A015820743069
:101430008A01582069308A0158206A308A01582070
:1014400064308A01582031308A0158203A308A01AC
:1014500058201730D0008A011F235108C100803066
:10146000A100C0308A011F200230A60041088A0175
:1014700027203A308A0158201830D0008A011F23D3
:101480005108C2008030A100C3308A011F20023001
:10149000A60042088A0127208A0186221730D2003E
:1014A0004108D3008A0131231830D2004208D3000A
:1014B0008A0131238A0115208030A1008A011F2072
:1014C00053308A01582027308A0158206D308A0114
:1014D00058206F308A01582072308A0158206730B6
:1014E0008A01582065308A0158206E308A015820C0
:1014F00073308A01582020308A0158206C308A01CC
:10150000582069308A01582063308A015820683099
:101510008A01582074308A0158203F308A015820AF
:101520008030A100C0308A011F2020308A0158205D
:101530008A0158208A0158208A0158208A0158209F
:101540008A0158204A308A01582061308A01582087
:1015500020308A0158208A0158208A0158208A01A7
:1015600058208A0158208A0158208A0158208A016F
:1015700058200130C3008A15051AEE2A8030A100D8
:10158000C0308A011F2020308A0158208A0158204B
:101590008A0158208A0158208A0158208A0158203F
:1015A0004A308A01582061308A01582020308A014F
:1015B00058208A0158208A0158208A0158208A011F
:1015C00058208A0158208A0158208A015820013069
:1015D000C3008A15051AEE2A8A15E92A8A15851983
:1015E000202B8030A100C0308A011F2020308A01CA
:1015F00058208A0158208A0158208A0158208A01DF
:1016000058208A0158204E308A01582065308A01BE
:1016100058208A01582020308A0158208A015820F9
:101620008A0158208A0158208A0158208A015820AE
:101630008A015820C3018A158519202B8A151B2B76
:101640008A15851A2D2B8A15851A282B8A15232B86
:10165000C8308A0113218A152F2B8A15BB2A19300D
:10166000D2004308D3008A013123013043028A1596
:10167000031DD62C8A0115208030A1008A011F206D
:1016800049308A0158206E308A01582073308A010F
:10169000582063308A01582068308A015820613010
:1016A0008A0158206B308A01582065308A01582001
:1016B0006C308A01582074308A01582069308A01C0
:1016C00058206A308A01582064308A01582032300C
:1016D0008A0158203A308A0158202030D0008A01EF
:1016E0001F235108C1008030A100C0308A011F2093
:1016F0000230A60041088A0127203A308A0158208A
:101700002130D0008A011F235108C2008030A1007F
:10171000C3308A011F200230A60042088A01272018
:101720008A0186222030D2004108D3008A01312369
:101730002130D2004208D3008A0131238A011520CA
:101740008030A1008A011F2055308A01582069305D
:101750008A01582074308A01582020308A0158208C
:101760006D308A01582065308A01582074308A0112
:10177000582020308A0158204C308A0158204430AB
:101780008A01582052308A0158203F308A0158205F
:101790008030A100C0308A011F2020308A015820EB
:1017A0008A0158208A0158208A0158208A0158202D
:1017B0008A0158204A308A01582061308A01582015
:1017C00020308A0158208A0158208A0158208A0135
:1017D00058208A0158208A0158208A0158208A01FD
:1017E00058208A15051A242C8030A100C0308A01A7
:1017F0001F2020308A0158208A0158208A01582051
:101800008A0158208A0158208A0158204A308A01CA
:10181000582061308A01582020308A0158208A01DE
:1018200058208A0158208A0158208A0158208A01AC
:1018300058208A0158208A0158200130C3008A1597
:10184000051A242C8A151F2C8A158519562C8030D0
:10185000A100C0308A011F2020308A0158208A014F
:1018600058208A0158208A0158208A0158208A016C
:1018700058204E308A01582065308A0158208A014C
:10188000582020308A0158208A0158208A01582087
:101890008A0158208A0158208A0158208A0158203C
:1018A000C3018A158519562C8A15512C8A15851A5B
:1018B000632C8A15851A5E2C8A15592CC8308A012A
:1018C00013218A15652C8A15F12B2430D200430888
:1018D000D3008A013123C3088A15031DD62C8A013F
:1018E00015208030A1008A011F2055308A01582020
:1018F00069308A01582074308A01582073308A0177
:10190000582063308A01582068308A01582061309D
:101910008A0158206B308A01582065308A0158208E
:101920006C308A01582074308A01582069308A014D
:1019300058206A308A01582064308A015820323099
:101940008A0158203A308A0158202230D0008A017A
:101950001F235108C1008030A100C0308A011F2020
:101960000230A60041088A0127203A308A01582017
:101970002330D0008A011F235108C2008030A1000B
:10198000C3308A011F200230A60042088A012720A6
:101990008A0186222230D2004108D3008A013123F5
:1019A0002330D2004208D3008A0131238A01432B1D
:1019B0008A0115208030A1008A011F2020308A0171
:1019C00058204C308A01582044308A015820523027
:1019D0008A01582020308A01582061308A0158201D
:1019E00066308A01582073308A01582074308A0189
:1019F000582065308A0158206C308A0158208A01AD
:101A0000582065308A0158206E308A0158202030D5
:101A10008A0158208A0158208A15851F3D2D803063
:101A2000A100C0308A011F2020308A0158208A017D
:101A300058208A0158208A0158208A0158208A019A
:101A400058206C308A01582069308A015820633050
:101A50008A01582068308A01582074308A01582041
:101A600020308A0158208A0158208A0158208A0192
:101A700058208A0158208A156A2D8030A100C03074
:101A80008A011F2020308A0158208A0158208A01AB
:101A900058208A0158208A01582064308A01582031
:101AA0006F308A0158206E308A0158206B308A01CD
:101AB000582065308A01582072308A015820203021
:101AC0008A0158208A0158208A0158208A0158200A
:101AD0008A0158208A15851A772D8A15851A722D44
:101AE0008A156D2DC8308A0113218A15792D8A1522
:101AF0000C2D8A01432B63008A157B2D8A157E2DC0
:02400E00503F21
:00000001FF
